:020000040000FA
:0400000035EF02F0E6
:040008000EEF00F007
:080018004FEF00F09EA221EF62
:1000200000F09E92A82BA8B1110000EE80F010EE17
:1000300093F00A0EA76FFF0ED76EFF0ED66ED58E09
:1000400011009EA029EF00F0829E819ECD909E908F
:100050001100E61C8116E61C8216D59EF294A707B5
:10006000EE1CD76EEE1CD66EA753D8B41100D58EF9
:100070000000828E818EFF0ECF6E390ECE6E9E9066
:10008000CD80000000000000000000000000000023
:1000900000000000E6508112E550821211001000AD
:1000A000A69CA69EA19865C0A8FF64C0A9FFA684CF
:1000B000550EA76EAA0EA76EA682A1A85DEF00F04E
:1000C000A6941200A69CA69E64C0A9FFA680A8CFF5
:1000D00065F01200080E616F62AF829A62BF828A79
:1000E0000000808A809A6237612F6CEF00F0120066
:1000F000948A080E616F626BD890623782BA62810F
:10010000808A809A612F7DEF00F0949A1200809887
:10011000450E626F6AEC00F078EC00F062C0A9F066
:1001200078EC00F062C068F078EC00F062C069F032
:1001300078EC00F062C06AF078EC00F062C06BF01E
:1001400078EC00F062C071F078EC00F062C070F002
:1001500078EC00F062C073F078EC00F062C072F0EE
:1001600078EC00F062C075F078EC00F062C074F0DA
:1001700078EC00F062C077F078EC00F062C076F0C6
:1001800078EC00F062C079F078EC00F062C078F0B2
:1001900078EC00F062C07BF078EC00F062C07AF09E
:1001A00078EC00F062C07DF078EC00F062C07CF08A
:1001B00078EC00F062C07FF078EC00F062C07EF076
:1001C000808812008098000E626F6AEC00F0000ECA
:1001D000626F6AEC00F080888098060E626F6AECAD
:1001E00000F0540E626F6AEC00F0750E626F6AECFC
:1001F00000F0C50E626F6AEC00F02A0E626F6AECC6
:1002000000F080888098460E626F6AEC00F078EC0F
:1002100000F062C068F078EC00F062C069F078EC41
:1002200000F062C06AF078EC00F062C06BF0808889
:10023000060EF76ECE0EF66EFF0E636F330E606F16
:10024000632B0900F528FCE0809863C062F06AEC3B
:1002500000F0F5CF62F06AEC00F08088602F20EFAC
:1002600001F08098020E626F6AEC00F0010E626F7E
:100270006AEC00F080888098020E626F628D6AECF2
:1002800000F0000078EC00F0808862B13BEF01F0F4
:100290008098240E626F6AEC00F0130E626F6AECB5
:1002A00000F080888098260E626F6AEC00F03B0EAA
:1002B000626F6AEC00F0808880980F0E626F6AECC3
:1002C00000F0000E626F6AEC00F080888098020EE9
:1002D000626F6AEC00F0020E626F6AEC00F08088D8
:1002E0008098020E626F628D6AEC00F0000078EC7C
:1002F00000F0808862B370EF01F080980F0E626F9B
:100300006AEC00F0A00E626F6AEC00F080888098C2
:10031000020E626F6AEC00F0020E626F6AEC00F08F
:1003200080888098020E626F628D6AEC00F0000097
:1003300078EC00F0808862B391EF01F08098250E90
:10034000626F6AEC00F0080E626F6AEC00F0808861
:100350001200676B8098A00E626F6AEC00F08088D4
:100360008098F00E626F6AEC00F0808880980F0E23
:10037000626F6AEC00F0000E626F6AEC00F0808839
:100380008098C00E626F6AEC00F08088B190270EF2
:10039000B36EB31E100EB26EB21EA192B180A1A2B6
:1003A000CFEF01F067B5829C67A5828C82A0DEEF5B
:1003B00001F0672FC6EF01F00DEF02F08098000EFC
:1003C000626F628D6AEC00F0000078EC00F08088CB
:1003D00062BBAAEF01F062BDAAEF01F087EC00F06A
:1003E000646B68C065F050EC00F0642B69C065F088
:1003F00050EC00F0642B6AC065F050EC00F0642B08
:100400006BC065F050EC00F068C06CF069C06DF036
:100410006AC06EF06BC06FF01200646B62EC00F0AB
:1004200065C06CF0642B62EC00F065C06DF0642B6D
:1004300062EC00F065C06EF0642B62EC00F065C009
:100440006FF01200902F2FEF02F0100E906F070E3A
:10045000F76E020EF66E9151F626D8B0F72A090013
:10046000F504666F9251665F1200D38CD38AD388ED
:10047000806A816A826A828C949C80889298828A3F
:10048000949A809A929A939C939A93989494949223
:1004900094989496939E949E7E6A7F6A000E936FC2
:1004A000000E946F400E956F000E966F200E976FA2
:1004B000000E986F100E996F000E9A6F000E9B6FD2
:1004C000040E9C6F000E9D6F020E9E6F000E9F6FBC
:1004D000080EA06F800EA16F000EA26F000EA36F1A
:1004E000800EA46F000EA56F000EA66F000EA46F05
:1004F000D56AD580F294F28ACD6ACD88CD8A9E9055
:100500009D809F80F90ECB6ECA6ACA8CCA86CA8249
:100510009E929D829F82F28CF28EB16AB18EB18AD8
:10052000A192DC0E816F836F856F876F896F8B6FF0
:100530008D6F8F6F050E806F826F846F866F886FEF
:100540008A6F8C6F8E6FCA84B190270EB36EB31E04
:10055000100EB26EB21EA192B180A1A2ADEF02F058
:10056000E2EC00F00000A9EC01F08098460E626F0A
:100570006AEC00F078EC00F0620E686F78EC00F046
:10058000620E696F78EC00F0620E6A6F78EC00F032
:10059000620E6B6F80886C39F00B916F010E906F5B
:1005A0006C390F0B926F090E9265D8EF02F0926FC3
:1005B00022EC02F08098A00E626F6AEC00F0808856
:1005C0008098F00E626F6AEC00F0808880980F0EC1
:1005D000626F6AEC00F066C062F06AEC00F080883E
:1005E0008098C00E626F6AEC00F08088B190070EB0
:1005F000B36EB31ED00EB26EB21EA192B180A1B284
:1006000062EF03F082B0FFEF02F08098000E626F9D
:10061000628D6AEC00F0000078EC00F0808887ECD6
:1006200000F06C516863FFEF02F06D516963FFEFFA
:1006300002F06E516A63FFEF02F06F516B63FFEFE0
:1006400002F0828CF29E70C080F071C081F0F28E58
:1006500000000000F29E72C082F073C083F0F28E40
:1006600000000000F29E74C084F075C085F0F28E28
:1006700000000000F29E76C086F077C087F0F28E10
:1006800000000000F29E78C088F079C089F0F28EF8
:1006900000000000F29E7AC08AF07BC08BF0F28EE0
:1006A00000000000F29E7CC08CF07DC08DF0F28EC8
:1006B00000000000F29E7EC08EF07FC08FF0F28EB0
:1006C000D8EF02F0829C22EC02F0D8EF02F0FF4259
:1006D000001400FFFF0000000001210500509E4BA8
:1006E0000002162B1200628080000A32C30F13C36F
:1006F00000FF00003B001747800301451800010F71
:10070000FF000A5A14641E6E287832823C8C46968A
:1007100050A0A05096468C3C823278286E1E6414FD
:100720005A0A0A5A50A0146446961E6E3C8C2878C9
:100730003282823278288C3C6E1E96466414A05019
:100740005A0A28780A5A50A014641E6E3C8C3282D1
:100750004696964682328C3C6E1E6414A0505A0A0D
:10076000782850A028780A5A1E6E3C8C3282469611
:1007700014646414964682328C3C6E1E5A0A7828A1
:10078000A05050A046963C8C28780A5A32821E6EA1
:10079000146464146E1E82325A0A78288C3C964681
:1007A000A05046963C8C50A028780A5A1E6E328281
:1007B0001464641482326E1E5A0A7828A0508C3C4D
:1007C000964646960A5A3C8C146450A028781E6EB1
:1007D000328282326E1E7828A05064148C3C5A0AF1
:1007E000964646960A5A50A03C8C28781E6E328255
:1007F0001464641482326E1E78288C3CA0505A0A0D
:0208000096461A
:020000040030CA
:03000100080914D7
:02000500800079
:0600080003C003E0034009
:0200000400F00A
:040000004D434850D4
:00000001FF
